:20000000855503A6B608002A03BDC2348501270536BDC254328502270536BDC2143285405F
:20002000270536BDAD6F328504270536BDDF1E328510270536BDC2A13285202703BDBC8D5E
:20004000B6080285E02703BDC0A3965885032708BDC5AFBDC377254A965985042708BDE2AF
:2000600009BDC37724F2BDC3772537965985202705BDFD88202CB60802841FBA0803BA08DF
:20008000012606965985022705BDBEBF201485102710B60802841FBA0801BA080326EABD9F
:2000A000C8873BD6592B30D67F582B2B54D77F969B2624BDC0DB96A12720D65954250EBDBB
:2000C000C531BDF2E5965984DF9759200D8641BDC428BDF2E52003B6380A397F00A1B608F1
:2000E0000284E0F6380A85602725D645C5042616CE0271092710F608002B14F6380B53C403
:20010000601127EF2009C6018520260150D7A139965984FD97597F005BD645C5082624B679
:2001200008029A6C976CC6345AC12F27074624F8D75B20F4965B270BBDC49196598A02974B
:200140005920058630BDC44BD645C50826587F005B966C85102710C688D75B7D006A2707FC
:20016000C61DF728102000B608019A6B976BC688CE280A5AC17F2713094624F7D75B7D004C
:200180006A27F0C61DE700D65B20E8965B271781812608D66BC52027028682BDC491965924
:2001A0008A02975920058680BDC44B7F005BB608039A6D976DC68FCE280A5CC198271309D9
:2001C0004624F7D75B7D006A27F0C61AE700D65B20E8965B272BBDC49196598A0297599638
:2001E000F2B73801B6300496F3B73801B6300596F4B73801B6300696F5B73801B6300720E1
:20020000058690BDC44BCE0116B6080085CC26030926F63996592B1BF60803C511261448EE
:200220002B11BDCBC196598A409759B728218699BDC49139B638067F0049BDDED9861DB79C
:2002400028014FB71000CE7A12F608002BF80926F87EF85CB6080997538502260EB638048D
:20026000B63808D659C4F7D7592035967E2A06BDDE7E7F007E960B84DF970B96F68A089764
:20028000F6B73008860BB73002CE0800FF3000D659CA08D7598609BDC491B63804BDFC6518
:2002A00039967F482B1596592B11D658582B0C969B2710D646C460C16027037EC3554F9711
:2002C0009B979DD646C5402643960B850226EC5D2B64D65954255FD654C510265DD659C423
:2002E000DFD759D654CEC359E500260D0808080808088CC37726F1205C5F08442508085CFE
:20030000C10526F7204FE6002B2C2002C60AD75B5FB608069BA02A03C68040375F915B2D6A
:20032000055C905B20F7D7A197A0324D2A137000A17000A0200B864120028642BDC4282029
:200340001196A127104FBDC428967F847F977FBDC531BDF2E5B608073908010001010104A3
:20036000FF0001030502FF0001020520FF0001020A01030002020A967B442569B608002766
:200380006985C3272085C2265CB608099753D6598502264DB63804B63808C4F7D759B60831
:2003A00000853C2745D67F582B1C8510270B960B85022731F608072031BDFA6AB1C6B02611
:2003C00024BDBCEA2021F608078520271DBDFA6AB1C6B02612BDAD5785202709BDBCEA20CE
:2003E00006C50826B90D39B608050C39960184EF9701960284EF9702960384EF9703960477
:2004000084EF97048620BDC44B8625BDC44B8623BDC44BBDD2B1BDD9A3965985082605BD93
:20042000BE862003BDFC6539D6862B0F91872714978796532A14BDADED200FD6532A0536BC
:20044000BDADED324D27037F007039D6862A41BDC4EE16CE0087A6002736BDC4EE11270821
:20046000088C009026F020286F008C008F271AA601A700088C008F26F64F978F97869687F3
:200480002707BDC4EE8A80978696532A03BDADED399187275136BDC4EE1696862A41847F1D
:2004A00011273C2A0FCE008EA600A701098C008626F6202BCE0088A6002711BDC4EE112788
:2004C0000B230E088C009026EE32201A32A70020153216A600E700088C009026F5200732C1
:2004E0009787CA80D78696532A03BDADED39375F4D273B81202733812527308123272D81DB
:200500000927238199271E812923238133231E81732716817923178188230D8189230F81E9
:2005200097230420095C5C5C5C5C5C5C5C5C17333996A13696542B2844251144251344250C
:200540001544251744271CBDDD542017BDE11A2015BDD60F200DBDD4022008BDCD4B2006E8
:20056000BDE03A322007324D2603BDC56E39967F2B2796594425069670260F201CBDF2E5AA
:200580008D18965984FE9759200C367F0070BDF2E58D07329770BDF2E539B60800260FBD26
:2005A000FA6AB1C65027F32305B1C65C23EC39965985042703BDE2099658D646582B084490
:2005C000240DCE0190200B442405CE03E82003CE0960B608008583262EBDFA6AC6FFD7A168
:2005E000B1C64D2707B1C65F2705201B7000A10926E0BDC531BDF2E596588A019758B6083F
:20060000008550260820A8D658C4FCD7587F00A1F608053901BDB302CA5D03CA5104CA45CB
:2006200005BDFA06C6B107BD2011C88712CA6113CA5514CA4915BE2016C6C017BD4822C911
:200640000E23C90624C8FE25C8F626C92027C93B32CC2933CC3134CC3935CC4136CC5A372E
:20066000C94142CA5943CA4D44CA4145CA3E46BDC150C70251C74152C9E853C9EE54C9F4C1
:2006800055C9FA56CA0060C6E761C72562C99563C99B64C9A165C9A766C9AD71C78672EFA3
:2006A000C173EF9A74C76775BE5E76CB5B77BE66708D17964585202626D746D7547EC7AAFC
:2006C0008D08D75454D7467EC7AABDC804D653C440270658965497563986503131200286CF
:2006E00056BDC4287EC7AABDC80486048D72CA01D70096018520272A84DF9701BDD3467E7C
:20070000C7A7BDC80486028D57CA02D70096028520270F84DF97028623BDC44BBDD4787E68
:20072000C7A47EC7AABDC80486108D34CA04D7009601852026748A2097018625BDC44B202B
:2007400066BDC80486208D18CA08D7009602852026588A2097028620BDC44BBDD7992044B5
:200760009754D600C4F039BDC8049654C601D754442504967F2A33960C8540272D84BF97F2
:200780000CBDE11A2024BDC8049654C608D75485082604967F2A13960C2A0F847F970CBD9E
:2007A000CD4B2006BDD6F0BDD2B1BDFC6539BDFC082545BDD9A3BDF415B608062A0540C6BE
:2007C000DF2002C6DDF72819C610816323035C8064F72801C61081092305800A5C20F78AEE
:2007E00010B72803F72802B6080084EF2607B60802856027C4F608073900000000000000BA
:00000001FF
